:05076500C103011F00AB
:0B08A400D2A0D2A1D2A2D2B6D2B722BD
:10024600E5A0F470030203117F057E001208AFE5F6
:10025600A0F47003020314E51E6401600302031494
:10026600F51EE5A0F430E012D2037F641208C54300
:1002760080F0C284E51F7002C2A4E5A0F430E1124A
:10028600D2037F461208C54380F0C285E51F70027F
:10029600C2A4E5A0F430E212D2037F281208C543B7
:1002A60080F0C286E51F7002C2A4E5A0F430E30F19
:1002B600751F01D203E4FF1208C54380F0C287E52B
:1002C600A0F430E410751F01D203D200D2A9D28C5B
:1002D60043B00EC2B1E5A0F430E514751F02D20397
:1002E60075270F7528A0D2A9D28C43B00EC2B2E5ED
:1002F600A0F430E619751F03D20375271F75284031
:10030600D2A9D28C43B00EC2B38003751E0175A06C
:01031600FFE7
:0103170022C3
:0B08AF00EF1FAC0670011E4C70F6221B
:1007C600E4F52FD2A77F08FE1208AFC2A77F507E9E
:1007D600001208AFD2A77F0E7E001208AF7F147EEC
:0407E600000208AF56
:02082800AD071A
:10082A007B08C2A7ED1392A77F057E001208AFD2FC
:07083A00A7EDC313FDDBEB8A
:010841002294
:10080A00E4FB7D08C2A7EBC313FBD2A730A70343BF
:0D081A0003807F087E001208AFDDE9AF0308
:0108270022AE
:1005EB00E4F9FFFBFAF52EF52DF52CF52BC2AF1226
:1005FB0007C67FCC1208287F441208287F057E008F
:10060B001208AF1207C67FCC1208287FBE1208282B
:10061B0012080AA90712080AD2AFEF7B00FAAF0142
:10062B00EB2FFBE43AFAAD03FCE4120129E4FBFAED
:10063B007920783F12001E1201627C037DE81201C3
:10064B00E3AA04AB057C007D0AAF03AE021201E303
:01065B00227C
:0B08BA00D2A3D2A4D2A5C2A6C2832202
:0308C5008F1D2262
:06000300E4F51DD2B0225D
:10084200758911758C3C758AB0D2A9D28C758D3C94
:0A085200758BB0D2ABD28ED2AF226C
:03001B0002079742
:10079700C0E0C0D0C28E758DFF758BF6D28EE52472
:1007A700C394644003752400E524D3951D50073096
:0F07B7000004D2B08002C2B00524D0D0D0E0320E
:03000B000204529A
:10045200C0E0C0F0C0D075D000C000C004C005C06C
:1004620006C007C28C758CFC758A18D28CC3E51C39
:100472009528E51B9527400EE51F64016008751B52
:1004820000751C00B200051CE51C7002051BE5226C
:10049200452170117521FF7522FF4380F0C287FF4D
:1004A2001208C58029E522F47003E521F4601FE5F6
:1004B20022152270021521AE21AF227C037DE812A3
:1004C20001E3EF65257001EE60048F25D203D007AA
:0F04D200D006D005D004D000D0D0D0F0D0E0328A
:1003BC007374617475733A20204E4F2057696E64C4
:1003CC00000000000000000000000000000073743A
:1003DC00617475733A204F7264696E6172790000B2
:1003EC000000000000000000000000007374617445
:1003FC0075733A20204E61747572616C00000000B8
:10040C00000000000000000000007374617475733C
:10041C003A20202020536C6565700000000000001D
:10042C0000000000000000007374617475733A20C2
:10043C00202020206175746F000000000000000077
:06044C00000000000000AA
:10076A000F08323727632020202020202020202035
:05077A00000217001B46
:100719001208757F8012000EE4F53074082530F850
:10072900E6FF1208987F321208670530E530C39456
:100739001040E87FC012000EE4F530E53075F01E78
:10074900A424BCF582E43403AF821208987F3212E4
:0B07590008670530E530C3941040E055
:010764002272
:0B085C00C2817F02120867D2827F0277
:0D086700EFD3940040077E6EDEFE1F80F38D
:010874002261
:0C000E008F90C282C28012085CC2822265
:0C0898008F90C282D28012085CC28222C3
:100875007F0112000E7F3F12000E7F0F12000E7FC8
:040885000602000E59
:10065C00AE17AF187C007D0A1201E3EF2430F508C9
:10066C00AE17AF187C007D0A1201E3ED2430F509BA
:10067C00C3E52194004039E522F47003E521F460D0
:10068C002FAE21AF227C037DE81201E3AA06AB0753
:10069C007C007D0A1201E3EF2430F5127C007D0A08
:1006AC00AF03AE021201E3ED2430F513751473227F
:0A06BC00751220751320751420221A
:1006C6001208757F8012000E12065CE4F519740894
:1006D6002519F8E6FF1208980519E519C394104084
:1006E600ED7FC012000EE4F519E51F75F01EA42477
:1006F600BCF582E43403F583E5822519F582E435F9
:1007060083F583E493FF1208980519E519C394103D
:0307160040D722A7
:10077F00C100012400022700000221FFFFC1010177
:07078F002500C10201230453
:10031800758911758DFF758BF6758CFC758A18D2E9
:10032800AFD2ABD28E751D32D200C288D2A81200CD
:1003380003C2871205EB8F261205EB8E298F2AC37D
:10034800E52A9432E52994004020E52A9518FFE52E
:10035800299517FED3EF9402EE9400500D4380F0D8
:10036800C287E4FF1208C51207EAE518652A700477
:10037800E51765296013C3E52A9450E529940050D0
:1003880008D203852917852A183003051206C6C224
:100398000320B60312088920B707B2027F051208A6
:1003A80067300206751F0412056D7F051208671273
:0403B80002468084F5
:1007EA00E4F52BF52CB2837F05120867052CE52C5E
:0F07FA007002052BC39414E52B6480948040E6B5
:0108090022CC
:0F08890074882522F52274133521F521D203221C
:10056D00AF267E00EF2402FDEE33FCC3E5189DE5BA
:10057D00179C402D851826E523D3940140021523A1
:10058D00E523B40103C2A022E523B40203C2A122D4
:10059D00E523B40303C2A222E5236404703FC2A382
:1005AD0022EF24FEFFEE34FFFED3E5189FE5179EE4
:1005BD00502B851826E523C3940450020523E5230B
:1005CD00B40103C2A022E523B40203C2A122E52394
:0E05DD00B40303C2A222E523B40402C2A32287
:10001E00EC4D6011E8497017ED33EC3304600DE4DC
:10002E00FCFFFEFD22E933E8330470F80201CE1224
:10003E00019958046009E4CC248150062850090225
:10004E0001D82840030201D5C0E0EB4A7044B980C4
:10005E0006D0E0FB0201C4EF4E701CBD8008EBFF22
:10006E00EAFEE9FD80EBE98DF0A4FEE5F002010762
:10007E00E9CDF9EAFEEBFFEF89F0A4FCE5F0CE89BD
:10008E00F0A42EFFE435F0CD89F0A42DFEE435F07A
:10009E008067EF4E7005BD80D780C3EF8BF0A4ACA8
:1000AE00F0EE8BF0A42CFCE435F0F8EF8AF0A42CE3
:1000BE00E5F038FCE433CB8DF0A42CFCE5F03BF8F6
:1000CE00EE8AF0A42CFCE5F038F8E433CF89F0A4E6
:1000DE002CFCE5F038CF3400CE89F0A42FFFE5F0EC
:1000EE003EFEE433C98DF0A42EFEE5F039CD8AF044
:1000FE00A42FFFE5F03EFEE43DFD33D0E0FB5007BC
:10010E000BBB000F0201D8EC2CFCEF33FFEE33FEDD
:06011E00ED33FD0201B00B
:1001240075F020800E75F010800575F0087D007E56
:10013400007F003392D530D503120238EC334010DF
:10014400EF33FFEE33FEED33FDEC33FCD5F0ED225F
:0E015400E5F0247EA2D513CC92E7CDCEFF229B
:10016200EDD2E7CD33EC3392D524814006E4FFFE95
:10017200FDFC22FCE4CFCECDCC24E0501174FF80F4
:10018200EDC3CC13CCCD13CDCE13CECF13CF047091
:07019200F030D5DE02023857
:10019900E9D2E7C933E833F892D5EDD2E7CD33ECAC
:0701A90033FC5002B2D52225
:1001B000EC30E7100FBF000C0EBE00080DBD0004B0
:1001C0000BEB6014A2D5EB13FCED92E7FD2274FF5C
:1001D000FCFDFEFF22E480F8A2D574FF13FC7D80B5
:0301E000E480EFC9
:030000000204E116
:0C04E100787FE4F6D8FD75813002052814
:1001E300BC000BBE0029EF8DF084FFADF022E4CC00
:1001F300F875F008EF2FFFEE33FEEC33FCEE9DECC9
:10020300984005FCEE9DFE0FD5F0E9E4CEFD22ED0E
:10021300F8F5F0EE8420D21CFEADF075F008EF2F58
:10022300FFED33FD4007985006D5F0F222C398FD49
:050233000FD5F0EA22E6
:0E023800C3E49FFFE49EFEE49DFDE49CFC22D7
:1004ED00020318E493A3F8E493A34003F68001F20A
:1004FD0008DFF48029E493A3F85407240CC8C33310
:10050D00C4540F4420C8834004F456800146F6DFDE
:10051D00E4800B0102040810204080900765E47E02
:10052D00019360BCA3FF543F30E509541FFEE493D3
:10053D00A360010ECF54C025E060A840B8E493A39A
:10054D00FAE493A3F8E493A3C8C582C8CAC583CAC5
:10055D00F0A3C8C582C8CAC583CADFE9DEE780BE7D
:010796000062
:00000001FF
